:030000000297E381
:03000300021312D3
:03000B00020BB530
:0300330002081CA4
:03004300020A00AE
:03005B0002833BE2
:10037000907FE9E070030204731470030204E72421
:10038000FE700302054F24FB700302046414700323
:1003900002045214700302043A1470030204492444
:1003A00005600302059E907FEBE024FE601614605A
:1003B000362402707B7412907FD4F07400907FD545
:1003C000F00205A5907FEAE0FF120A99EA49600D64
:1003D000EA907FD4F0E9907FD5F00205A5907FB434
:1003E000E04401F00205A5907FEAE0FF120A58EA16
:1003F00049603312A23BF54E907FEEE0FFE54ED30D
:100400009F4003E0F54EE54ED394404003754E40C7
:10041000AE02AF017C7F7D00AB4E129137907FB56D
:10042000E54EF00205A5907FB4E04401F00205A579
:10043000907FB4E04401F00205A5907F00E521F033
:10044000907FB57401F00205A5907FEAE0F52102E6
:1004500005A5907FEAE0F535D202438810D2EBD2B1
:10046000A80205A5907F00E535F0907FB57401F0F6
:100470000205A5907FE8E0247F6024146031240207
:10048000705BA200E433FF25E0FFA205E4334F9048
:100490007F00F0E4A3F0907FB57402F00205A5E4BC
:1004A000907F00F0A3F0907FB57402F00205A59054
:1004B0007FECE0F45480FFC4540FFFE054072F2575
:1004C000E024B4F582E4347FF583E05401907F00AA
:1004D000F0E4A3F0907FB57402F00205A5907FB41C
:1004E000E04401F00205A5907FE8E024FE601D24B1
:1004F0000260030205A5907FEAE0B40105C2000294
:1005000005A5907FB4E04401F00205A5907FEAE0E4
:100510007034907FECE0FF5407FEF54EEF30E703B8
:10052000434E10907FD7E54EF0E54E4420F0EFF4B7
:100530005480FDC4540F2E25E024B4F582E4347FAA
:10054000F583E4F0805F907FB4E04401F080569042
:100550007FE8E024FE60182402704A907FEAE0B44D
:100560000104D200803F907FB4E04401F0803690D7
:100570007FEAE07020907FECE0F45480FFC4540FD9
:10058000FFE054072F25E024B4F582E4347FF5839F
:100590007401F08010907FB4E04401F08007907FF8
:0C05A000B4E04401F0907FB4E04402F0AD
:0105AC00222C
:1005AD00754AFF7549FF75480F754700D203C2069E
:1005BD00C202C200C205C2019003007419F0E4909A
:1005CD0001BCF0C2049001C0F0A3F0C2AFC2A812EA
:1005DD000C22E49002AFF09001BDF0900100F0A369
:1005ED00F0A3F0A3F0A3F0A37410F0A37401F0A393
:1005FD007408F07E017F001219C1754C12754D0AF9
:10060D0090010BE0FF054DE54DAC4C7002054C140F
:10061D00F5828C83EFF090010CE04480FF054DE5F1
:10062D004DAC4C7002054C14F5828C83EFF09001AB
:10063D000DE0FF054DE54DAC4C7002054C14F582F7
:10064D008C83EFF090010EE0FF054DE54DAC4C7045
:10065D0002054C14F5828C83EFF090120AE493FF9F
:10066D0074019390011CCFF0A3EFF090011CE0FFFB
:10067D00A3E0FEEF6EFF90011CF0A3E06FFFF09082
:10068D00011CE06FF0E0FEA3E0FFE4FCFD755210ED
:10069D007553027554127555AC129426754C12751E
:1006AD004DB290010DE0FF054DE54DAC4C700205CE
:1006BD004C14F5828C83EFF090010EE0FF054DE5B3
:1006CD004DAC4C7002054C14F5828C83EFF0907F8D
:1006DD0092E0FFC4540F2441FF054DE54DAC4C7025
:1006ED0002054C14F5828C83EFF0054DE54DAE4CB3
:1006FD007002054C14F5828E83E4F07582107583BB
:10070D0001E0FCA3E0FDA3E0FEA3E0FF90011812C1
:10071D00A3EE7E017F181286BE900118E0FCA3E0C7
:10072D00FDA3E0FEA3E0FF75520A75530675541242
:10073D007555B8129426D2E843D820907FAB74FF3C
:10074D00F05391EF907FAFE04401F0907FAEE04425
:10075D001FF0D2AF20012E20012BA2039207120908
:10076D00C575465075456D7544337543002001E4DC
:10077D007FFF7EFF7DFF7CFF784312A3D7EC4D4EAC
:10078D004F60D180E8300105120370C20130060AB6
:10079D001209FB5003120AE8C20612965E9001BDC3
:1007AD00E0600C129201E49001BDF0907FD3F090C7
:1007BD0002AFE0B40F031299B912A095E4FF7401D2
:1007CD00A807088002C333D8FCFE9001BCE05E6030
:1007DD001474282FF8E6D3940A40047E0180027E1B
:1007ED00008E4B8003754B0174682FF582E4342025
:1007FD00F583E54BF00FBF04C5E52CD3940A4004F7
:0E080D007F0180027F0090206CEFF0020792C6
:01081B0022BA
:04081C0053D8EF328C
:10082000E533C39401400E907F93E04430F0907F15
:1008300095E044C0F07FF47E011209AE907F96E00F
:1008400054FEF07F0A7E001209AE907F96E04408C5
:10085000F07F057E001209AE907F96E054FBF07F9A
:10086000057E001209AEE533C39401500E7F027D70
:10087000FF1282EA7F057E001209AE907F96E04467
:1008800002F0E0547FF07F057E001209AE907F9663
:10089000E04440F07F057E001209AE907F96E05460
:1008A000BFF07F327E001209AE907F96E04440F0A8
:0808B0007F327E001209AE2226
:1008B800907F96E054FDF0E04480F07F0A7E0012BD
:1008C80009AEE533C39401500E7F02E4FD1282EABB
:1008D8007F057E001209AE907F96E054BFF07F0539
:1008E8007E001209AE907F96E04404F07F057E00FA
:1008F8001209AE907F96E054F7F07F057E0012094A
:10090800AE907F96E04401F07F057E001209AEE5C7
:1009180033C39401400E907F93E054CFF0907F95BD
:08092800E0543FF0120B002225
:10093000900AF4E4937076907F937430F0907F94F3
:10094000743CF0907F9574C6F07F0A7E001209AE69
:10095000E4907F9CF0907F967408F0907F9C74CF19
:10096000F07F0A7E001209AE902070E0FFC4540FA1
:10097000F533C394015007907F96E04480F0E490F3
:100980007F97F0907F9D7402F0E533C39401400B94
:10099000E4907F98F0907F9E74C0F0907FE2741294
:0E09A000F01208207582F475830A74FFF022AD
:1009AE008E5D8F5EE55E155EAE5D7002155D4E600E
:0709BE00051209EA80EE2298
:1009C500907FD6E054FBF0E04408F0300704E044A3
:1009D50002F07FD07E071209AE907FD6E054F7F083
:0509E500E04404F022D3
:1009EA007400F58690FDA57C05A3E582458370F920
:0109FA0022DA
:0509FB001208B8D32230
:100A0000020C4E00020C8100020C6600020CC000B9
:100A1000020CAA00020AED00020AEE00020AEF0030
:100A2000020CDB00020DCB00020D1700020E2B00A2
:100A3000020D5300020E8B00020D8F00020EEB0020
:100A4000020AF000020AF200020AF100020AF300B0
:080A5000020F4B00020F6100D0
:020A58008F4FBE
:100A5A00E4F5507551FF75521275536AAB51AA529B
:100A6A00A95390000112A254B4031DAF500550EFD0
:100A7A00B54F012212A23B7E0029FFEE3AA9077563
:0E0A8A0051FFF552895380D47B007A00790029
:010A9800223B
:100A9900E4FE7551FF755212755312AB51AA52A952
:100AA9005390000112A2546402702DAD060EEDB5EB
:100AB90007012290000212A2AD85F04FF550624F56
:100AC900E54F6250E550624F29FDE54F3AA905759A
:0E0AD90051FFF552895380C37B007A007900EB
:010AE70022EC
:050AE800120820D322DA
:010AED0032D6
:010AEE0032D5
:010AEF0032D4
:010AF00032D3
:010AF10032D2
:010AF20032D1
:010AF30032D0
:030AF400000407F4
:090B0000907FD6E04480F080747F
:100B7D00438701000000000000000000000000227B
:100B8D00538EF7E58954F14401F589758CB1D2A9DD
:100B9D0075984075CBFF75CAF375C834E4FF7F05B2
:070BAD007828E4F608DFFCE4
:010BB400221E
:100BB500C0E0C083C082C0D075D000C000C006C0F0
:010BC5000728
:100BC600300416758CF8758A307F2FAE071FEE60DD
:100BD6003C9020007455F080F2758CB17F28EFD3DD
:100BE600942C5009A807E66001160F80F1900300C7
:100BF600E0600214F09001C0E07002A3E0600E9085
:0D0C060001C1E024FFF09001C0E034FFF0D8
:0F0C1300D007D006D000D0D0D082D083D0E0322E
:100C2200D200758E10120930E533C394014008904A
:100C32007F927402F08005E4907F92F0128000129D
:0C0C42000F7D1294F7121B0C120B8D2278
:100C4E00C0E0C083C082D2015391EF907FAB74019C
:080C5E00F0D082D083D0E03217
:100C6600C0E0C083C082907FC4E4F05391EF907FD0
:0B0C7600AB7404F0D082D083D0E032D9
:100C8100C0E0C083C0825391EF907FAB7402F090BB
:100C91007FD8E0700D907FD9E07007E52C70037567
:090CA1002C14D082D083D0E03283
:100CAA00C0E0C083C0825391EF907FAB7410F0D044
:060CBA0082D083D0E0327D
:100CC000C0E0C083C082300202D2065391EF907F11
:0B0CD000AB7408F0D082D083D0E0327B
:100CDB00C0E0C083C082C0D075D0105391EF907F1D
:100CEB00A97402F0E53430E013E53230E0079020D0
:100CFB0004E04401F0902001E04401F0E52C700386
:0C0D0B00752C14D0D0D082D083D0E03200
:100D1700C0E0C083C082C0D075D0105391EF907FE0
:100D2700A97404F0E53430E113E53230E10790208F
:100D37000CE04401F0902009E04401F0E52C700339
:0C0D4700752C14D0D0D082D083D0E032C4
:100D5300C0E0C083C082C0D075D0105391EF907FA4
:100D6300A97408F0E53430E213E53230E20790204D
:100D730014E04401F0902011E04401F0E52C7003ED
:0C0D8300752C14D0D0D082D083D0E03288
:100D8F00C0E0C083C082C0D075D0105391EF907F68
:100D9F00A97410F0E53430E313E53230E307902007
:100DAF001CE04401F0902019E04401F0E52C7003A1
:0C0DBF00752C14D0D0D082D083D0E0324C
:100DCB00C0E0C083C082C085C084C086758600C069
:100DDB00D075D0105391EF907FAA7402F0E53420B8
:100DEB00E006907FC7F08022E53130E00A907FC7A4
:100DFB00E09002F8F08013E52230E007902004E049
:100E0B004402F0902001E04402F0E52C7003752CB5
:100E1B0014D0D0D086D084D085D082D083D0E0328D
:100E2B00C0E0C083C082C085C084C086758600C008
:100E3B00D075D0105391EF907FAA7404F0E5342055
:100E4B00E106907FC9F08022E53130E10A907FC93D
:100E5B00E09002F9F08013E52230E10790200CE0DE
:100E6B004402F0902009E04402F0E52C7003752C4D
:100E7B0014D0D0D086D084D085D082D083D0E0322D
:100E8B00C0E0C083C082C085C084C086758600C0A8
:100E9B00D075D0105391EF907FAA7408F0E53420F1
:100EAB00E206907FCBF08022E53130E20A907FCBD7
:100EBB00E09002FAF08013E52230E207902014E074
:100ECB004402F0902011E04402F0E52C7003752CE5
:100EDB0014D0D0D086D084D085D082D083D0E032CD
:100EEB00C0E0C083C082C085C084C086758600C048
:100EFB00D075D0105391EF907FAA7410F0E5342089
:100F0B00E306907FCDF08022E53130E30A907FCD70
:100F1B00E09002FBF08013E52230E30790201CE009
:100F2B004402F0902019E04402F0E52C7003752C7C
:100F3B0014D0D0D086D084D085D082D083D0E0326C
:100F4B00C0E0C083C0825391EF907FA97480F0D032
:060F5B0082D083D0E032D9
:100F6100C0E0C083C0825391EF907FAA7480F0905B
:0C0F710001BD74FFF0D082D083D0E032CC
:100F7D0090012012A3FA000025809001247408F03E
:100F8D00A37401F0A3746EF0A3F0A37413F0A37413
:100F9D0011F0E4A3F0A3F090011EF090011EE0FF0C
:100FAD0004A3F0EF75F00DA42401F9740335F0A836
:100FBD0001FC7D017B017A01791F7E007F0D12A25C
:100FCD00127E017F1F1287A690011EE004F0E0C380
:100FDD00940440C7E4F52790011EF090011EE0FF38
:100FED00C39404501A74F82FF582E43402F583E4A7
:100FFD00F074232FF8E4F690011EE004F080DCE499
:10100D00F534E5C0602F90011E7401F090011EE0D3
:10101D00FFD39404501FEF14FF7401A8070880023A
:10102D00C333D8FC42347E017F1E12844190011ED1
:10103D00E004F080D7E4F53EF522F531F53290016C
:10104D001EF090011EE0FF75F008A42406F582E461
:10105D003420F583E054F0FE74C52FF582E434019D
:10106D00F583EEF0743A2FF8A60674362FF8E4F6F1
:10107D00742D2FF8E4F674FC2FF582E43402F58319
:10108D00E4F090011EE004F0E0B404B6902060E0BE
:04109D00540FF54EA9
:1010A1007003021126E490011EF090011EE0FFC3BF
:1010B100940450E47401A807088002C333D8FC5596
:1010C1004E605A90011EE0FE75F008A42402F582DC
:1010D100E43420F583E0FFEE75F008A42405F582E1
:1010E100E43420F583E0EE75F008A42406F582E4EB
:1010F1003420F583E0FFAF06EE75F00DA42402F570
:1011010082E43403F583E0FCA3E0FDA3E0FEA3E069
:10111100F5668E658D648C637D061283DF90011EFA
:06112100E004F0808522CD
:02112700AC0713
:10112900907FA5E04480F0EC25E04441907FA6F053
:101139007B3CAF031BEF7016907FA5E04440F09015
:101149007FA6E0FD7D32AF051DEF60D480F8907F6A
:10115900A5E0FD30E0DC20E109E04440F07EFF7FBE
:10116900F922ED30E20C907FA5E04440F07EFF7F4C
:10117900FA22907FA5E04420F0907FA6E0FD7B1E37
:10118900AF031BEF7016907FA5E04440F0907FA657
:10119900E0FD7D32AF051DEF608680F8907FA5E008
:1011A900FD20E0DC7B3CAF031BEF7019907FA5E0CD
:1011B9004440F0907FA6E0FD7D32AF051DEF70033E
:1011C90002112980F5907FA5E0FD30E0D930E209D0
:1011D900E04440F07EFF7FFA22C2AF907FA5E04451
:0C11E90040F0907FA6E0FDD2AFFF7E003A
:0111F50022D7
:1012000012010001FFFFFF401007018042000102B0
:10121000030109025800010104803C090400000A8E
:10122000FFFFFF050705810240000007050102409E
:10123000000007058202400000070502024000008E
:101240000705830240000007050302400000070570
:1012500084024000000705040240000007058702E1
:1012600040000007050702400000040309042403AE
:1012700043006F006E006E00650063007400200084
:101280005400650063006800200049006E006300A0
:101290002E001803570068006900740065004800BC
:1012A0004500410054002D0034001A035800580036
:1012B0002D00580058002D005800580058005800C4
:1012C000580058002A0343006F006E006600690052
:1012D0006700750072006100740069006F006E00A5
:1012E000200053007400720069006E006700220342
:1012F00049006E00740065007200660061006300C2
:101300006500200053007400720069006E006700E1
:021310000000DB
:10131200C0E0C0F0C083C082C085C084C086C0D097
:1013220075860075D018902060E0540FF5F07011AA
:10133200D0D0D086D084D085D082D083D0F0D0E0F7
:101342003275860010F00B10F11210F21910F32012
:1013520080D4E528700375281402137CE5297003F4
:1013620075291402150DE52A7003752A1402169EBA
:10137200E52B7003752B1402182F902002E0543FC6
:1013820020E23A20E10B20E40B20E514600902136D
:1013920043021465021343438204E0F53A02134305
:1013A200438204E0432D010213435382F843820532
:1013B200E042365382FBE054FBF002134330E10279
:1013C20080E8F585E53230E00A5382F8438204E092
:1013D20054FEF0E58520E3569020507400F09020F2
:1013E200587401F0907FE2E04440F0907FE305867C
:1013F200907E800586E585F0A3E584F00586907FE2
:10140200E5E53FFD030303FEF0F0F0F0F0F0F0F04D
:10141200DEF6907FE2E054BFF09020587400F09026
:101422007FB7EDF0902001E054FEF00213437F40BD
:10143200907E800586902000E584FE2405FD8D8443
:10144200E08E8430E009E00586F0A30586DFEF0533
:1014520086C374409F907FB7F00586A3E054FEF0E8
:10146200021343532DFAE5236008752300D2E7FEE9
:10147200800A907FC7E0FE70030214FF9020507430
:1014820000F09020587401F0907FE2E04440F09028
:101492007FE30586907E400586E585F0A3E584F02E
:1014A2000586907FE5EE30E7080586E02438F005F2
:1014B20086EE547FFE5407FBEE547860300303033C
:1014C20030E30474077B08FDFCE0E0E0E0E0E0E0EC
:1014D200E0DDF6EBFE6019EC640770118B23907F60
:1014E200E2E054BFF09020587400F0801BE0DEFD73
:1014F200907FE2E054BFF09020587400F0902001F9
:10150200E054FDF0907FC7F002134390200AE054AC
:101512003F20E23A20E10B20E40B20E514600902AF
:1015220013430215F6021343438204E0F53B021310
:1015320043438204E0432E010213435382F8438261
:1015420005E042375382FBE054FBF002134330E1E3
:101552000280E8F585E53230E10A5382F8438204DD
:10156200E054FEF0E58520E3569020507401F0909F
:1015720020587401F0907FE2E04440F0907FE30550
:1015820086907E000586E585F0A3E584F0058690C9
:101592007FE5E540FD030303FEF0F0F0F0F0F0F02C
:1015A200F0DEF6907FE2E054BFF09020587400F035
:1015B200907FB9EDF0902009E054FEF00213437FD2
:1015C20040907E000586902008E584FE2405FD8D6E
:1015D20084E08E8430E009E00586F0A30586DFEF23
:1015E2000586C374409F907FB9F00586A3E054FE40
:1015F200F0021343532EFAE5246008752400D2E763
:10160200FE800A907FC9E0FE70030216909020507F
:101612007401F09020587401F0907FE2E04440F0B1
:10162200907FE30586907DC00586E585F0A3E5847D
:10163200F00586907FE5EE30E7080586E02438F075
:101642000586EE547FFE5407FBEE547860300303A8
:101652000330E30474077B08FDFCE0E0E0E0E0E037
:10166200E0E0DDF6EBFE6019EC640770118B24906C
:101672007FE2E054BFF09020587400F0801BE0DE5F
:0E168200FD907FE2E054BFF09020587400F01D
:10169000902009E054FDF0907FC9F00213439020A0
:1016A00012E0543F20E23A20E10B20E40B20E51445
:1016B0006009021343021787021343438204E0F5D3
:1016C0003C021343438204E0432F0102134353823D
:1016D000F8438205E042385382FBE054FBF00213EA
:1016E0004330E10280E8F585E53230E20A5382F8C2
:1016F000438204E054FEF0E58520E35690205074C8
:1017000002F09020587401F0907FE2E04440F090A5
:101710007FE30586907D800586E585F0A3E584F06E
:101720000586907FE5E541FD030303FEF0F0F0F050
:10173000F0F0F0F0DEF6907FE2E054BFF090205839
:101740007400F0907FBBEDF0902011E054FEF002A9
:1017500013437F40907D800586902010E584FE2411
:1017600005FD8D84E08E8430E009E00586F0A30558
:1017700086DFEF0586C374409F907FBBF00586A38C
:10178000E054FEF0021343532FFAE5256008752557
:1017900000D2E7FE800A907FCBE0FE7003021821A2
:1017A0009020507402F09020587401F0907FE2E095
:1017B0004440F0907FE30586907D400586E585F006
:1017C000A3E584F00586907FE5EE30E7080586E026
:1017D0002438F00586EE547FFE5407FBEE54786003
:1017E0003003030330E30474077B08FDFCE0E0E012
:1017F000E0E0E0E0E0DDF6EBFE6019EC640770117C
:101800008B25907FE2E054BFF09020587400F08068
:101810001BE0DEFD907FE2E054BFF09020587400A2
:10182000F0902011E054FDF0907FCBF00213439034
:10183000201AE0543F20E23A20E10B20E40B20E59F
:10184000146009021343021918021343438204E08F
:10185000F53D021343438204E04330010213435336
:1018600082F8438205E042395382FBE054FBF002E8
:10187000134330E10280E8F585E53230E30A538214
:10188000F8438204E054FEF0E58520E356902050B2
:101890007403F09020587401F0907FE2E04440F02F
:1018A000907FE30586907D000586E585F0A3E584BD
:1018B000F00586907FE5E542FD030303FEF0F0F0BE
:1018C000F0F0F0F0F0DEF6907FE2E054BFF0902010
:1018D000587400F0907FBDEDF0902019E054FEF0B8
:1018E0000213437F40907D000586902018E584FE1A
:1018F0002405FD8D84E08E8430E009E00586F0A3A8
:101900000586DFEF0586C374409F907FBDF0058696
:10191000A3E054FEF00213435330FAE52660087545
:101920002600D2E7FE800A907FCDE0FE7003021908
:10193000B29020507403F09020587401F0907FE230
:10194000E04440F0907FE30586907CC00586E58505
:10195000F0A3E584F00586907FE5EE30E708058684
:10196000E02438F00586EE547FFE5407FBEE5478F1
:10197000603003030330E30474077B08FDFCE0E000
:10198000E0E0E0E0E0E0DDF6EBFE6019EC6407701B
:10199000118B26907FE2E054BFF09020587400F045
:1019A000801BE0DEFD907FE2E054BFF09020587491
:1019B00000F0902019E054FDF0907FCDF002134329
:0119C00032F4
:0419C100AD07AC06BC
:1019C5007906ED2404F582E43CF583E0FAA3E0FB17
:1019D5004A7003021B09E9B407004003021ADB90B1
:1019E50019EBF8282873021AB9021A71021A5A0259
:1019F5001A40021A2F021A1A021A00907FA5E04413
:101A050080F08D828C83A3E0FF25E044A0907FA623
:101A1500F019021ADB198D828C83E0C39420400AE9
:101A2500A3A3E0907FA6F0021ADB8D828C83A3A38B
:101A3500E0A3E0907FA6F019021ADB907FA5E044B1
:101A450080F08D828C83A3E0FF25E044A1907FA6E2
:101A5500F019021ADBEB64014A7008907FA5E04497
:101A650020F019907FA6E0F55919806AED2404F558
:101A750082E43CF583E0FEA3E064024E7008907FAB
:101A8500A5E04420F019907FA6E0FFED2406F5823D
:101A9500E43CF583E475F00112A29785F082F583A5
:101AA500EFF0ED2404F582E43CF58374FFF5F012C4
:101AB500A2818022907FA5E04440F0907FA6E0FFC0
:101AC500ED2406F582E43CF583E0FAA3E0F5828A8D
:101AD50083EFF07F0822907FA5E0F55930E0F730DD
:101AE500E207E04440F07F0622E9D3940250030266
:101AF50019C7E55930E1030219C7907FA5E04440B5
:061B0500F07F07227F08BB
:011B0B0022B7
:101B0C00E533C39401501C7F057E001209AE7F02A1
:101B1C007DFF1282EA7F057E001209AE7F037DFFF6
:041B2C001282EA2215
:108000007BFF7A12791B90000412A254FD8B5075ED
:108010005112755224E4907FE1F0907FE0F0F54E2C
:10802000F54F9002AEF0907FDFF0907FDEF0907F12
:10803000A974FFF0907FAAF0E4FCEC25E024B4F5ED
:1080400082E4347FF583E4F00CBC10EEE4907FDD35
:10805000F0AF051DEF70030281C6AB50AA51A952C3
:1080600090000112A254640560030281B5900003E0
:1080700012A2546401600302813C90000212A254D7
:10808000FF547FFCD394075003028116ECC3941075
:108090004003028116EF30E742E54FAE4E7802CE44
:1080A000C313CE13D8F9FF74F02CF582E4347FF5B6
:1080B00083EFF0907FE0E0FFEC24F8FE7401A80667
:1080C000088002C333D8FC4F907FE0F09002AEE00E
:1080D00004F0907FDDE04480F0803EE54FAE4E78C6
:1080E00002CEC313CE13D8F9FF74E82CF582E43422
:1080F0007FF583EFF0907FE1E0FFEC24F8FE740160
:10810000A806088002C333D8FC4F907FE1F09002AC
:10811000AEE004F080037FFF2290000412A25425F9
:108120004FF54FE4354EF54E90000512A254FEE493
:10813000254FF54FEE354EF54E0281B8AB50AA51A2
:10814000A95290000312A254FF64026005EF640379
:10815000706090000212A254FF547FFCD394075029
:108160004EEF30E71E907FDEE0FF7401A804088028
:1081700002C333D8FCFE4F907FDEF0907FACE04E20
:10818000F08035907FDFE0FF7401A804088002C30F
:1081900033D8FCFE4F907FDFF0907FADE04EF0ECE7
:1081A00025E024C5F582E4347FF583ECF080097F77
:1081B000FF227FFF227FFF2274072552F552E4350C
:1081C00051F55102805120030D9002AEE0600790FE
:0881D0007FAEE04402F07F00E5
:0181D8002284
:0481D9008E598F5AD2
:1081DD00755B03E55A2404F582E43559F583E0FE19
:1081ED00A3E04E70030282E7E55B604E1460381425
:1081FD00602014600302828B907FA5E04480F0859F
:10820D005A82855983A3E0FF25E044A0907FA6F014
:10821D00806C855A82855983E0C394204009A3A3BD
:10822D00E0907FA6F08057155B855A82855983A310
:10823D00A3E0A3E0907FA6F08044E55A2406F582E2
:10824D00E43559F583E475F00112A29785F082F5B6
:10825D0083E0907FA6F0907FA5E04440F0E55A249E
:10826D0004F582E43559F58374FFF5F012A281858A
:10827D005A82855983A3A3E475F00112A281907FE0
:10828D00A5E0F55C30E0F730E207E04440F07F0612
:10829D0022E55C20E10A907FA5E04440F07F0722B3
:1082AD00E55B70317F017E001209AE907FA5E04441
:1082BD0080F0855A82855983A3E0FF25E044A09084
:1082CD007FA6F0907FA5E0F55C30E0F730E1D57545
:0C82DD005B030281E0155B0281E07F087A
:0182E9002272
:0282EA00AE07DD
:1082EC007C02EC14601514701E907FA5E04480F0A5
:1082FC00EE25E04440907FA6F0800C907FA6EDF038
:10830C00907FA5E04440F0907FA5E0FB30E0F8BC06
:10831C00020A20E107E04440F07F0722EB30E20A3A
:0E832C00907FA5E04440F07F0622DCB67F087B
:01833A002220
:10833B00C0E0C083C082C2A99003007419F0D2A917
:0F834B0053917F9001C4E4F0D082D083D0E03210
:10835A00EF75F008A42400F582E43420AB82FAF524
:10836A0083A3E4F08B828A83A3A3A3E0F56174BF9D
:10837A00F08B828A83A3A3E04410F08B828A83A3C2
:10838A00A3A3E4F08B828A83A3F0F9ED601D740144
:10839A007E00A807088005C333CE33CED8F9FFE4A0
:1083AA00EF5531600479098002790D8B828A83A3A3
:1083BA00A3A374BFF08B828A83A3A3E054EFF08B4C
:1083CA00828A83A3A3A3E561F0AE02AF038F828EF4
:0483DA0083A3E9F0A0
:0183DE00227C
:0483DF008F618D62BB
:1083E300E4F567743F2FF876087F807E257D007C57
:1083F30000AB66AA65A964A863D312A3B340267F22
:10840300007E967D007C00A863D312A3B3500C7545
:108413006740743F2561F87610800A756780743F62
:108423002561F87638E56745624401FFE56175F03B
:0D84330008A42402F582E43420F583EFF064
:018440002219
:108441008F828E83E014F557C3940440037FFF228B
:10845100E55775F008A42400F582E43420AF82F5D5
:10846100588F59E55725E024C6F582E4347FF5831A
:10847100E020E10FE55725E024C7F582E4347FF5DC
:1084810083E4F074232557F8E4F6E5592404F582D2
:10849100E43558F583E04403F0E55775F00DA42465
:1084A10002F582E43403F583E0FCA3E0FDA3E0FEE2
:1084B100A3E0F5668E658D648C637D06AF571283EC
:1084C100DFAF577D0112835A855982855883A3A353
:1084D100E020E043E0FFE5592405F582E43558F555
:1084E10083E0E5592406F582E43558F583E0FFE59C
:1084F1005775F00DA42402F582E43403F583E0FC02
:10850100A3E0FDA3E0FEA3E0F5668E658D648C63B8
:108511007D06AF571283DF74F82557F582E43402E4
:10852100F583E4F0E55725E0FFC3740C9F75F04037
:10853100A42440F582E5F0347BAF82FEE55725E0C7
:1085410024EFF582E43402F583EEF0A3EFF0AF57A8
:0F8551007401A807088002C333D8FC42347F00AE
:0185600022F8
:108561008F828E83E014F557C3940440037FFF226A
:10857100AF57E4FD12835A74F82557F582E43402AB
:10858100F583E4F0E55775F008A42400F582E4349E
:1085910020AF82F5598F5AF583E5822404F582E4F0
:1085A1003583F583E054FCF0E55775F00DA4240CF8
:1085B100F582E43403F583E4F0E55775F00DA42466
:1085C10002F582E43403F583E0FCA3E0FDA3E0FEC1
:1085D100A3E0F5668E658D648C637D06AF571283CB
:1085E100DFE55A2405F582E43559F583E030E009E9
:1085F100855A82855983E0F558AF577401A8070859
:108601008002C333D8FCF45234E55725E024C6F583
:1086110082E4347FF583E020E10FE55725E024C7AC
:0B862100F582E4347FF583E4F07F0075
:01862C00222B
:04862D008E578F587D
:108631008F828E83E014F559C3940440037FFF2297
:10864100E55975F008A42401F582E43420F583E0AE
:1086510054037066855882855783A3E030E028E58E
:108661005975F00DA42402F582E43403F583E0FC8E
:10867100A3E0FDA3E0FEA3E0F5668E658D648C6347
:108681007D02AF591283DF855882855783A3E0307D
:10869100E128E55975F00DA42402F582E43403F5CF
:1086A10083E0FCA3E0FDA3E0FEA3E0F5668E658D0B
:0C86B100648C637D04AF591283DF7F00EE
:0186BD00229A
:1086BE008F828E83C083C082E0FDA3A3A3E0FCED76
:1086CE006CD082D083F08F828E83A3A3A3C083C08D
:1086DE0082E0FD8F828E83E0FCED6CD082D083F041
:1086EE008F828E83C083C082A3A3A3E0FDEC6DD0E6
:1086FE0082D083F08F828E83A3C083C082E0FD8FF1
:10870E00828E83A3A3E0FCED6CD082D083F08F82A7
:10871E008E83A3A3C083C082E0FD8F828E83A3E0ED
:10872E00FCED6CD082D083F08F828E83A3C083C089
:10873E0082E0FD8F828E83A3A3E0FFED6FD082D007
:03874E0083F02293
:04875100AD07AC06BE
:10875500790D8D828C83E014FEC3940440037FFF62
:10876500228C578D58EE75F00DA42401F582E43462
:1087750003AF82FEAD0119ED60240FEFAC06700169
:108785000E14F5828C83E0FD0558E558AA57700252
:10879500055714F5828A83E06D60D97F01227F0039
:0187A50022B1
:0487A6008E578F5803
:1087AA008F828E83E014F55EC3940440037FFF2218
:1087BA00E55E75F008A42400F582E43420AF82F562
:1087CA005F8F60855882855783A3E0FCA3E0FDA3F1
:1087DA00E0FEA3E0FF7B087A0079007800D312A3B9
:1087EA00B34010855882855783A312A3FA0000006C
:1087FA0008802E855882855783A3E0FCA3E0FDA359
:10880A00E0FEA3E0FF7B007A0879077800C312A391
:10881A00B3500E855882855783A312A3FA0007081E
:10882A0000855882855783A3E0F8A3E0F9A3E0FA0C
:10883A00A3E0FB7F007E507D467C0012A3218F5C63
:10884A008E5B8D5A8C597B0A7A007900780012A3C4
:10885A0021AF038F5DAF5CAE5BAD5AAC597B0A7A30
:10886A00007900780012A3218F5C8E5B8D5A8C5997
:10887A00E55DC394054015E55C2401F55CE4355BD0
:10888A00F55BE4355AF55AE43559F5598560828520
:10889A005F83A3E4F0856082855F83A3A3A3E0449A
:1088AA0080F0856082855F83E55CF0AF5CAE5BAD8E
:1088BA005AAC59780812A3C4856082855F83A3EFF6
:1088CA00F0856082855F83A3A3A3E0547FF0E4F57B
:1088DA005DE558240BF582E43557F583E0FF30E077
:1088EA00235401F0E5602404F582E4355FF583E062
:1088FA0054FDF0AF5E7401A807088002C333D8FCA8
:10890A004222803674017E00A85E088005C333CEF9
:10891A0033CED8F9FFE4EF5522601FE5602404F551
:10892A0082E4355FF583E04402F0AF5E7401A80784
:10893A00088002C333D8FCF45222E5582408F58291
:10894A00E43557F583E0FFB46205435D0A801AEF08
:10895A00B47205435D088011EFB47405435D02806B
:10896A0008EF646E60037FFF22E558240BF582E46A
:10897A003557F583E0FF30E303435D80EF30E712BC
:10898A00435D40E5602404F582E4355FF583E04405
:10899A0002F0E558240BF582E43557F583E030E11F
:1089AA0020AF5E7401A807088002C333D8FC4232A4
:1089BA00E5602404F582E4355FF583E04401F08044
:1089CA0010AF5E7401A807088002C333D8FCF452C2
:1089DA0032E558240BF582E43557F583E0FF30E49D
:1089EA0011AE5E7401A806088002C333D8FC423176
:1089FA008010AE5E7401A806088002C333D8FCF466
:108A0A005231EF20E10330E403E4F55D85608285AD
:108A1A005F83A3A3A374BFF0856082855F83A3A34A
:108A2A00E4F0E55DF0E558240AF582E43557F5836C
:108A3A00E0FFE5602404F582E4355FF583EFF0E5B5
:108A4A0058240AF582E43557F583E0FFE5602405EA
:108A5A00F582E4355FF583EFF0E5582409F582E401
:108A6A003557F583E0FFE5602406F582E4355FF5C6
:108A7A0083EFF0E5582409F582E43557F583E0FFE2
:108A8A00E5602407F582E4355FF583EFF0856082BF
:108A9A00855F83A3A3A3E4F0856082855F83A3A394
:108AAA00F0855882855783A3E0FCA3E0FDA3E0FE8E
:108ABA00A3E0F5668E658D648C637D06AF5E1283D6
:108ACA00DF755D08E558240CF582E43557F583E037
:108ADA006003435D10E5602404F582E4355FF583A5
:108AEA00E05403455DF0E5582405F582E43557F571
:108AFA0083E0FEC394054006EED3940840037FFF4B
:108B0A0022E5582406F582E43557F583E0FDC3943F
:108B1A00014006EDD3940240037FFF22ED14FF25A6
:108B2A00E025E0FFEE24FB4FF55DE5582407F582CA
:108B3A00E43557F583E024D0601814601A24C36022
:108B4A001E146009240A7014435D188012435D08DC
:108B5A00800D435D388008435D2880037FFF2285AE
:108B6A006082855F83A3A3A3E55DF074017E00A8FC
:108B7A005E088005C333CE33CED8F9FFE4EF55340F
:108B8A006007AF5E7D0112835AAA57A9587B01C0BC
:108B9A0003C001E55E75F00DA42401F9740335F0F4
:108BAA00A801FCAD03D001D0037E007F0D12A212F2
:028BBA007F003A
:018BBC002296
:108BBD008F828E83E014FEC3940440037FFF22EE68
:108BCD0075F008A42400F582E43420AD82FC9001F8
:108BDD002C7408F0EE04A3F0E4A3F08D828C83E5F1
:108BED00822406F582E43583F583E090012FF08D24
:108BFD00828C83E5822405F582E43583F583E05488
:108C0D001E900130F0742D2EF8E6A3F0AF0674011E
:108C1D00A807088002C333D8FCF557E533C3940188
:108C2D00400D902078E0540F755800F55980097F5C
:108C3D00021211278E588F59C3E5586480948040D5
:108C4D00DAE5575559900132F07E017F2C7D0712E0
:048C5D00916A7F0099
:018C610022F0
:108C62008F828E83E014FEC3940440037FFF22EEC2
:108C720075F008A42400F582E43420AF82FE90014E
:108C820033740AF08F828E83E5822404F582E43500
:108C920083F583E0900134F07E017F337D021291EF
:038CA2006A7F00E6
:018CA50022AC
:048CA6008E578F58FE
:108CAA008F828E83E014FEC3940440037FFF22EE7A
:108CBA0075F008A42400F582E43420AD82FC8558BE
:108CCA0082855783A3E0600FED2404F582E43CF526
:108CDA0083E04402F08043EE75F00DA4240CF58283
:108CEA00E43403F583E030E020EE25E024C6F58283
:108CFA00E4347FF583E030E1F07F60ED2405F5820E
:108D0A00E43CF583E05FB507F2AE04AF05EF240457
:0C8D1A00F582E43EF583E054FDF07F009C
:018D2600222A
:048D2700AD07AC06E2
:108D2B008D828C83E014FEC3940440037FFF22EEFC
:108D3B0075F008A42400F582E43420AF82FE8D8206
:108D4B008C83A3E0600FEF2404F582E43EF583E00F
:108D5B004401F0800DEF2404F582E43EF583E054EA
:048D6B00FEF07F0097
:018D6F0022E1
:048D7000AD07AC0699
:108D74008D828C83E014FEC3940440037FFF22EEB3
:108D840075F008A42400F582E43420AF82FE8D82BD
:108D94008C83A3E0600D8F828E83A3A3A3E0444061
:108DA400F0800B8F828E83A3A3A3E054BFF07F00D7
:018DB400229C
:108DB5008F828E83E014FEC3940440037FFF22AFAD
:108DC500067401A807088002C333D8FC423E7F0021
:018DD500227B
:048DD6008E578F58CD
:108DDA008F828E83A3E0F55C8F828E83E0F559D370
:108DEA00940440037FFF22E55924FE601614601F95
:108DFA001460282403702E7E7E7F80755A7E755BF0
:108E0A008080227E7E7F00755A7E755B0080167E8A
:108E1A007D7F80755A7D755B80800A7E7D7F0075B7
:108E2A005A7D755B00E55C701B855B82855A83748D
:108E3A00FFF0E55925E024B5F582E4347FF5837423
:108E4A0001F08048E5582402FFE43557FEE55C60EE
:108E5A00230FEFAC0670010E14F5828C83E0FD053A
:108E6A005BE55BAA5A7002055A14F5828A83EDF013
:108E7A00155C80D9855882855783A3E0FFE559257B
:0E8E8A00E024B5F582E4347FF583EFF07F003D
:018E980022B7
:108E9900EF2405F558E43EF5579001357407F09035
:108EA900017A7401F0A37436F0855882855783A33B
:108EB900A3A3E0FEA3E08E59F55A8558828557830E
:108EC900E0249E606124F9600E24F17003028F7A18
:108ED90024146003028FC8855882855783A3E0FE56
:108EE900A3E0FFC3E49FF55C74019EF55BD3E55CE9
:108EF900943FE55B94004006755B00755C3FD3E5E4
:108F09005A955CE559955B5003028FCBAE5BAF5C1C
:108F1900855882855783A3A3A3EEF0FEA3EFF08EB5
:108F290059F55A028FCB855882855783A3E0FEA352
:108F3900E0FFC374309FF55CE49EF55BD3E55C9478
:108F490010E55B94004006755B00755C10D3E55A2B
:108F5900955CE559955B406AAE5BAF5C8558828547
:108F69005783A3A3A3EEF0FEA3EFF08E59F55A8021
:108F790051855882855783A3E0FEA3E0FFC3E49F90
:108F8900F55CE49EF55B455C600BD3E55C943FE5DD
:108F99005B94004006755B00755C3FD3E55A955CB0
:108FA900E559955B401CAE5BAF5C8558828557835C
:108FB900A3A3A3EEF0FEA3EFF08E59F55A80037F29
:108FC9000122855882855783E0249E700302908B85
:108FD90024F9605824F170030290DB241460030221
:108FE900911F855882855783A3E0FEA3E0FFD394A0
:108FF900FFEE9400400302911F900175EFF0E55ACE
:10900900155AAE59700215594E700302911F9001FD
:1090190075E0FF04F0A807E6FF90017AE475F00116
:1090290012A29785F082F583EFF080D28558828568
:109039005783A3E0FEA3E0FFC39480EE940050039E
:1090490002911FD3EF94FFEE9400400302911F9009
:109059000176EFF0E55A155AAE59700215594E705E
:109069000302911F900176E0FF04F0A807E6FF9044
:10907900017AE475F00112A29785F082F583EFF089
:1090890080D2855882855783A3E0FEA3E0FFC3946D
:1090990020EE9400500302911FD3EF942FEE940019
:1090A9005074900177EFF0E55A155AAE59700215D0
:1090B900594E6062900177E0FF04F0A807E6FF903F
:1090C900017AE475F00112A29785F082F583EFF039
:1090D90080D5855882855783A3E0FFA3E090017866
:1090E900CFF0A3EFF0E55A155AAE59700215594E53
:1090F9006024900178E475F00112A29785F082F559
:1091090083E0FF90017AE475F00112A29785F0825D
:10911900F583EFF080CF7E017F35855882855783AF
:0D912900A3A3A3E0A3E004FD12916A7F0060
:019136002216
:109137008E628F638C648D65AF031BEF60240563BC
:10914700E563AE627002056214F5828E83E0FF0567
:1091570065E565AC647002056414F5828C83EFF0F5
:0391670080D6228D
:06916A008D5DAB07AA06B3
:1091700075614075600D755F03755E00907FC2E09C
:1091800020E1F9AF61AE60AD5FAC5EEC4D4E4F706B
:1091900008907FC27402F080D7907FC2E020E11671
:1091A000AF03AE027C7B7D80AB5D129137907FC3B5
:0891B000E55DF07F01227F0064
:0191B8002294
:1091B900900184740BF0A3E533F0900AF5E49390E1
:1091C9000186F0900AF6E493900187F0E490017C1F
:1091D900F0A3F0A3F0A3F0A3F0A37410F0A374011B
:1091E900F0A37488F07E017F7C1219C17E017F840F
:0791F9007D1412916A7F0052
:01920000224B
:109201007E7B7F40754E7B754F40907FD3E0FF851D
:109211004E51854F52E5522401F556E43551F5552D
:10922100E4F550855282855183E0FE14B40C005060
:109231005B909239F828287302925D02925D029246
:109241006702927102927102927102928502925D9D
:1092510002927B02925D02928D02925DEF64026046
:109261002B7550FF8026EF640E60217550FF801C26
:10927100EF640360177550FF8012EF6403600D7592
:1092810050FF8008EF640660037550FFE5506015DC
:109291009001987411F0A3EEF07E017F987D021287
:1092A100916AAF5022E4F550855282855183E014D2
:1092B100B40F0040030293CF9092C0F828287302A4
:1092C10092ED0292F902930502935302935E029387
:1092D1006902937402937F02938A0293950293A089
:1092E1000293A70293CF0293B20293BDAF56AE553C
:1092F1001284418F500293D2AF56AE551285618FC1
:10930100500293D2855553855654E5542401FFE408
:109311003553FE1286BEAF54AE531287518F50EFB4
:10932100640160030293D2AF54AE531287A68F50EB
:10933100E55070030293D2855482855383E075F022
:109341000DA424F4F582E43402AF82FE1287A60252
:1093510093D2AF56AE55128CA68F508074AF56AED5
:1093610055128D278F508069AF56AE55128D708F73
:1093710050805EAF4FAE4E128E998F508053AF56D4
:10938100AE55128BBD8F508048AF56AE5512862D0B
:109391008F50803DAF56AE55128C628F5080321285
:1093A10091B98F50802BAF56AE55128DB58F50802D
:1093B10020AF56AE55128DD68F508015AF4FAE4EA1
:1093C1007C027DAF7B40129137E4F55080037550EC
:1093D100FFE550601D9001987411F085528285510E
:1093E10083E0900199F07E017F987D0212916AAF2E
:1093F1005022855282855183E0FF1424FA500424BF
:10940100FE701F9001987410F0A3EFF085568285CD
:109411005583E090019AF07E017F987D0312916A55
:049421008F50AF5069
:019425002224
:089426008F518E508D4F8C4ECA
:10942E0075580175599CE4F557AF531553EF7003FA
:10943E000294C4AF52E4FCFDFEF8F9FAAB07AF514B
:10944E00AE50AD4FAC4E12A321AF038F56AF51AEFF
:10945E0050AD4FAC4EC004C005C006C007AF52E4BD
:10946E00FCFDFEF8F9FAAB07D007D006D005D00404
:10947E0012A3218F518E508D4F8C4EE5562430F510
:10948E0056D39439400674072556F5560559E559B5
:10949E00AE587002055814F5828E83E4F00559E536
:1094AE0059AE587002055814F5828E83E556F005B4
:1094BE00570557029437E559155970021558AF578D
:1094CE001557EF6023E5591559AE5870021558F52A
:1094DE00828E83E0FF0555E555AC54700205541499
:0894EE00F5828C83EFF080D6BB
:0194F6002253
:1094F700E49001C9F07E017FCA9001BEEEF0A3EFB0
:0A950700F09001C2EEF0A3EFF02295
:10951100AA07A9059001C9E0C394405061AC027447
:10952100017E00A804088005C333CE33CED8F9FFED
:10953100E4EF55346045EA04FF9001C2E0FCA3E08A
:10954100FDF5828C83EFF0A3E9F08D828C83A3A3D8
:10955100EBF09001C2E475F00312A281FCD3E5F0B7
:109561009487EC9402400A9001C27401F0A374CA7A
:10957100F0C2AF9001C9E004F0D2AF7F01227F00B9
:0195810022C7
:109582009001C9E0D3940040559001BEE0FCA3E0F5
:10959200AA04F97B01C003C002C001AA06A907A858
:1095A20001AC02AD03D001D002D0037E007F0312D2
:1095B200A2129001BEE475F00312A281FCD3E5F081
:1095C2009487EC9402400A9001BE7401F0A374CA1D
:1095D200F0C2AF9001C9E014F0D2AF7F01227F0048
:0195E2002266
:1095E300907FC2E020E1737E7B7F8075537B75544F
:1095F30080E5542401FFE43553A9077B018B55F51E
:10960300568957FE129582EF6050AB55AA56A9575B
:1096130012A23B14FF90000112A254B40216C2AF6F
:10962300EF75F008A42401F582E43420F583E044C7
:1096330004F0D2AF74017E00A807088005C333CEBF
:1096430033CED8F9FFE4EF5534600F855482855348
:0A96530083740DF0907FC37404F0DF
:01965D0022EA
:10965E001295E3E4F54E743A254EF8E654F0F54FC4
:10966E0074C5254EF582E43401F583E0654FFFC4E1
:10967E00540FF550602274C5254EF582E43401F581
:10968E0083E54FF0AF4E7D01E54F4550FB1295112E
:10969E00EF70051295E380EC054EE54EC394044041
:1096AE00B51295E3E53E6048E4F54EAF4E7401A861
:1096BE0007088002C333D8FCF54F553E6029E54EAE
:1096CE0075F008A42405F582E43420F583E030E635
:1096DE0016AF4E7D047B80129511EF70051295E347
:1096EE0080EFE54FF4523E054EE54EC3940440BB69
:1096FE00900300E060030297DF7419F0E533C39422
:10970E0001400D902078E0540F755100F5528009FC
:10971E007F021211278E518F52C3E55164809480BF
:10972E0040DA9001BCE06552F06037E4F54EAF4E82
:10973E007401A807088002C333D8FCF54F9001BC12
:10974E00E0554F6014AF4E7D08E54F5552FB129514
:10975E0011EF70051295E380EC054EE54EC39404AF
:10976E0040CC9001BCE552F0E4F54EC2AF74362504
:10977E004EF8E6F54FE4F6D2AF534F1EE54F6011AB
:10978E00AF4E7D02AB4F129511EF70051295E3802F
:10979E00EF742D254EF8E6F54F74FC254EF582E458
:1097AE003402F583E0654F6011AF4E7D04AB4F126E
:1097BE009511EF70051295E380EF74FC254EF5823E
:1097CE00E43402F583E54FF0054EE54EC3940440B4
:0497DE009A1295E363
:0197E2002264
:0C97E300787FE4F6D8FD75816702982AB3
:1097EF000205ADE493A3F8E493A34003F68001F2DE
:1097FF0008DFF48029E493A3F85407240CC8C3337B
:10980F00C4540F4420C8834004F456800146F6DF49
:10981F00E4800B010204081020408090986FE47ED2
:10982F00019360BCA3FF543F30E509541FFEE4933E
:10983F00A360010ECF54C025E060A840B8E493A305
:10984F00FAE493A3F8E493A3C8C582C8CAC583CA30
:10985F00F0A3C8C582C8CAC583CADFE9DEE780BEE8
:10986F006024028A010204081020408081828488CB
:10987F0090A0C0C1C2C4C8D0E0E1E2E4E8F0F1F2C8
:08988F00F4F8F9FAFCFDFEFFFC
:0198970000D0
:089898008B598A5A895B8D5C33
:1098A000E4F55DF55EAF5C155CEF6036AB59055BCA
:1098B000E55BAA5A7002055A14F912A23BFFE55D56
:1098C000E55E6F25E0FFE433FE74952FF582EE34FC
:1098D0009EF583E55DFFE493F55D7401936FF55E9E
:0698E00080C3AE5DAF5E27
:0198E600225F
:0B98E700C0E0C083C082C0D075D01864
:1098F200902060E0540FFE30E005902002E0FFEE81
:1099020030E10590200AE0FFEE30E205902012E0FF
:10991200FFEE30E30590201AE0FF9001C4E0B51E8F
:0A99220004E4F080059001C4EEF0AB
:09992C00D0D0D082D083D0E0320B
:02993500A90384
:10993700EF75F008A42400F582E43420AB82FAE541
:109947005C455DF55EE960148A83E5822404F5824F
:10995700E43583F583E04DF0E4FE8013EB2404F552
:1099670082E43AF583E0FFEDF4FCEF5CF0AE5EEBEA
:109977002406F582E43AF583E0555EFCB50603AFAD
:109987000522E55C5CFEE55D5CFDE96016EE7004B2
:109997007F0180027F00AE07ED70047F0180027FA8
:1099A70000AD07EE6003AF5C22ED6003AF5D227F81
:0199B70000AF
:0199B800228C
:1099B9007555027556B0900335740FF0855682853A
:1099C9005583A3E0FF900337F0855682855583E0E0
:1099D900900336F090033874FFF0755703755839C2
:1099E900EF14B40B004003029E5D9099FAF8282801
:1099F90073029A1B029ABA029BBF029BDE029BDE8C
:109A0900029C94029CCF029CF4029DB2029DE20248
:109A19009E0EE4F54EE54E75F008A42400F582E4A7
:109A29003420AF82F5538F54E4FFE4FEEF601074E5
:109A39008A2EF582E43402F583E0F4F54F800D7443
:109A49008A2EF582E43402F583E0F54FE5542407C4
:109A5900F582E43553F583E54FF0E0F550654F6045
:109A690038E4900338F0E54E04FD0558E558AA5747
:109A79007002055714F5828A83EDF00558E558AC54
:109A8900577002055714F5828C83E54FF08558828B
:109A9900855783E550F0029E630EBE248F0FEF6455
:109AA900027087054EE54E64046003029A1E029E09
:109AB90063E4F54EAF4EE4FD12835A054EE54ED3ED
:109AC900940340F09000047498F0A374E7F0E4F56F
:109AD900507E207F00755320755400F54EAF4E74AB
:109AE90001A807088002C333D8FCF54F9001C4F0E0
:109AF9009001C0E4F0A3740AF0855482855383A3CE
:109B09007402F09001C4E0B54F349001C0E07002D6
:109B1900A3E070EF900338F0E54E04FF0558E558CF
:109B2900AC577002055714F5828C83EFF085588283
:109B390085578374FFF0E49001C4F07550FF9001DC
:109B4900C4E0FF6037E4900338F0E54E04FE0558A1
:109B5900E558AC577002055714F5828C83EEF00571
:109B690058E558AC577002055714F5828C83EFF00D
:109B7900855882855783E54FF07550FFE55070167B
:109B890074082554F554E43553F553054EE54E64F0
:109B9900046003029AE6E4F54EAF4E7D0112835A42
:109BA900054EE54ED3940340F09000047413F0A3DE
:109BB9007412F0029E63855682855583E014FF7402
:109BC90001A807088002C333D8FC9002F7F090017E
:109BD900C4F0029E639001C07403F0A374E8F0E43A
:109BE900F5509002F7E0FF9001C4E0B50719900124
:109BF900C0E07002A3E070EA900338F085588285CE
:109C0900578374FFF0F550E5506003029E6390019D
:109C1900C0F0A37496F09001C0E07002A3E070F662
:109C2900E533C39401400D902078E0540F7551003D
:109C3900F55280097F021211278E518F52C3E551C7
:109C49006480948040DAE552540FF5509002F7E0B1
:109C5900555070047F0180027F008F4F85568285A1
:109C69005583A3E0B4050CE54F70047F0180027FA2
:109C7900008F4FE54F7003029E63E4900338F0852F
:109C89005882855783E550F0029E63E4FFFD1283F5
:109C99005A7E207F00755320755400855482855360
:109CA90083A3A3A3E04480F0855482855383740180
:109CB900F0A3E4F0855482855383A3A3A3E0547FE2
:109CC900F0D204029E63C2047E207F007553207582
:109CD9005400E5542405F582E43553F583E030E674
:109CE900F1E4FF7D0112835A029E63E4F550F54EBB
:109CF900AF4EE4FD12835AE54E75F008A42400F531
:109D090082E43420AF82F5538F54F583E58224042D
:109D1900F582E43583F583E054FCF0AF4E7D017B99
:109D290001755C80755D401299358F50E550701151
:109D3900AF4E7D027B01755C10755D201299358FE0
:109D490050E5507010AF4E7D01FB755C80755D402C
:109D59001299358F50E5507010AF4E7D02FB755C3E
:109D690010755D201299358F50AF4E7D0112835ABF
:109D7900E5506026E4900338F0E54E04FF0558E508
:109D890058AC577002055714F5828C83EFF085584B
:109D990082855783E550F0029E63054EE54ED394C4
:109DA900035003029CF9029E63E4900359F0A3F067
:109DB900A3F0A3F0A3F0A37410F0A3749EF0A3740E
:109DC90085F07E037F591281D9EF64087003029EE2
:109DD90063E4900338F0029E63E4900359F0A3F022
:109DE900A3F0A3F0A3F0A37410F0A3E557F0A3E543
:109DF90058F07E037F591219C1EF6408605CE49042
:109E09000338F08055E5562402FFE43555FAA907D1
:109E19007B017D10129898EF4E7032900359F0A390
:109E2900F0A3F0A3F0A3F0A37410F0E55624029078
:109E39000360F0E4355590035FF07E037F5912818A
:109E4900D9EF64086014E4900338F0800DE49003BE
:109E590038F080069003387401F09001C0E4F0A353
:109E6900740AF09001C0E07002A3E070F67E037FEF
:0B9E7900357D2412916AE49002AFF0E6
:019E840022BB
:109E8500FFFEFCF8F0E0C080000103070F1F3F7FD5
:109E95000000C0C1C1810140C30103C00280C241AD
:109EA500C60106C00780C7410500C5C1C48104407D
:109EB500CC010CC00D80CD410F00CFC1CE810E402D
:109EC5000A00CAC1CB810B40C90109C00880C8413D
:109ED500D80118C01980D9411B00DBC1DA811A40AD
:109EE5001E00DEC1DF811F40DD011DC01C80DC417D
:109EF5001400D4C1D5811540D70117C01680D641AD
:109F0500D20112C01380D3411100D1C1D0811040BC
:109F1500F00130C03180F1413300F3C1F2813240AC
:109F25003600F6C1F7813740F50135C03480F4417C
:109F35003C00FCC1FD813D40FF013FC03E80FE412C
:109F4500FA013AC03B80FB413900F9C1F88138403C
:109F55002800E8C1E9812940EB012BC02A80EA41AC
:109F6500EE012EC02F80EF412D00EDC1EC812C407C
:109F7500E40124C02580E5412700E7C1E6812640AC
:109F85002200E2C1E3812340E10121C02080E041BC
:109F9500A00160C06180A1416300A3C1A2816240AC
:109FA5006600A6C1A7816740A50165C06480A4417C
:109FB5006C00ACC1AD816D40AF016FC06E80AE412C
:109FC500AA016AC06B80AB416900A9C1A88168403C
:109FD5007800B8C1B9817940BB017BC07A80BA41AC
:109FE500BE017EC07F80BF417D00BDC1BC817C407C
:109FF500B40174C07580B5417700B7C1B6817640AC
:10A005007200B2C1B3817340B10171C07080B041BB
:10A01500500090C191815140930153C052809241AB
:10A02500960156C057809741550095C1948154407B
:10A035009C015CC05D809D415F009FC19E815E402B
:10A045005A009AC19B815B40990159C0588098413B
:10A05500880148C0498089414B008BC18A814A40AB
:10A065004E008EC18F814F408D014DC04C808C417B
:10A07500440084C185814540870147C046808641AB
:10A08500820142C043808341410081C180814040BB
:10A09500E4FF74F82FF582E43402F583E0700302DF
:10A0A500A138743A2FF8E620E50302A138EF75F0E0
:10A0B50008A42400F582E43420AD82FCF583E58212
:10A0C5002405F582E43583F583E0546064607063AC
:10A0D500EF25E024EFF582E43402F583E475F00121
:10A0E50012A29785F082F583E08D828C83F074F857
:10A0F5002FF582E43402F583E014F07036EF25E0A5
:10A1050024C7F582E4347FF583E4F0EF25E0FEC350
:10A11500740C9E75F040A42440F582E5F0347BADC7
:10A1250082FCEF25E024EFF582E43402F583ECF0C0
:0CA13500A3EDF00FEF6404600302A0979C
:01A1410022FB
:10A14200E709F608DFFA8046E709F208DFFA803EFF
:10A1520088828C83E709F0A3DFFA8032E309F608EC
:10A16200DFFA8078E309F208DFFA807088828C8354
:10A17200E309F0A3DFFA806489828A83E0A3F60808
:10A18200DFFA805889828A83E0A3F208DFFA804CE2
:10A1920080D280FA80C680D4806980F280338010B9
:10A1A20080A680EA809A80A880DA80E280CA803322
:10A1B20089828A83ECFAE493A3C8C582C8CCC5839A
:10A1C200CCF0A3C8C582C8CCC583CCDFE9DEE7806A
:10A1D2000D89828A83E493A3F608DFF9ECFAA9F0E9
:10A1E200EDFB2289828A83ECFAE0A3C8C582C8CC3F
:10A1F200C583CCF0A3C8C582C8CCC583CCDFEADE58
:10A20200E880DB89828A83E493A3F208DFF980CCB9
:10A2120088F0ED2402B4040050C2F582EB2402B4AB
:10A22200040050B823234582F582EF4E60AEEF6002
:09A23200010EE5822390A1927354
:10A23B00BB010689828A83E0225002E722BBFE0221
:09A24B00E32289828A83E4932254
:10A25400BB010CE58229F582E5833AF583E02250BF
:10A2640006E92582F8E622BBFE06E92582F8E22209
:0DA27400E58229F582E5833AF583E4932223
:10A28100C5F0F8A3E028F0C5F0F8E5821582700268
:06A291001583E038F02205
:10A29700A3F8E0C5F025F0F0E5821582700215837A
:06A2A700E0C838F0E822D7
:10A2AD00BB0110E58229F582E5833AF583E0F5F0EF
:10A2BD00A3E0225009E92582F886F008E622BBFECC
:10A2CD000AE92582F8E2F5F008E222E5832AF58312
:08A2DD00E993F5F0A3E99322D7
:10A2E50075F008758200EF2FFFEE33FECD33CDCC30
:10A2F50033CCC58233C5829BED9AEC99E5829840B3
:10A305000CF582EE9BFEED9AFDEC99FC0FD5F0D68F
:10A31500E4CEFBE4CDFAE4CCF9A88222B800C1B9B9
:10A325000059BA002DEC8BF084CFCECDFCE5F0CBF7
:10A33500F97818EF2FFFEE33FEED33FDEC33FCEB30
:10A3450033FB10D703994004EB99FB0FD8E5E4F9EB
:10A35500FA227818EF2FFFEE33FEED33FDEC33FCD8
:10A36500C933C910D7059BE99A4007EC9BFCE99ACC
:10A37500F90FD8E0E4C9FAE4CCFB2275F010EF2F11
:10A38500FFEE33FEED33FDCC33CCC833C810D70711
:10A395009BEC9AE899400AED9BFDEC9AFCE899F84C
:0EA3A5000FD5F0DAE4CDFBE4CCFAE4C8F922DF
:10A3B300EB9FF5F0EA9E42F0E99D42F0E89C45F000
:01A3C3002277
:10A3C400E8600FECC313FCED13FDEE13FEEF13FF77
:03A3D400D8F1229B
:10A3D700080808E6CF2FF618E6CE3EF618E6CD3D7C
:07A3E700F618E6CC3CF6225B
:0CA3EE00ECF0A3EDF0A3EEF0A3EFF022E2
:10A3FA00A8828583F0D083D08212A41112A41112EC
:10A40A00A41112A411E473E493A3C583C5F0C58310
:10A41A00C8C582C8F0A3C583C5F0C583C8C582C8AC
:01A42A00220F
:00000001FF
